:10000000830100308A00042883010A128A11DD2F3F
:10001000820745344C3445344B34543452344934DB
:100020004B34003482077F34BF34DF34EF34F7348D
:06003000FB34FD34FE3438
:100F320083120313A1000430A2005330A300A30BB9
:100F4200A02FA20B9E2FA10B9C2F0800831203132C
:100F5200A100C92F66308600E330870008003B30CD
:100F62008600E33087000800E6308600DE30870026
:100F72000800EE308600F3308700080066308600F5
:100F82002E30870008003B308600EF3087000800D3
:100F92002108453A0319AB2F0C3A0319B02F023A34
:100FA2000319B52F073A0319BA2F1E3A0319BF2F97
:100FB200063A031D0800C42F831603138601870116
:100FC2008801FF308312880086008700A001FF306D
:100FD200880000308A00200808200A128A11A727F8
:100FE20000308A0020081220880001300A128A117B
:0E0FF2009927A00A083020020318E72FE82FE5
:02400E0071FF40
:00000001FF
